:0A00060000308A00C62800003F30D9
:100010008400000803191B280130F800F701F70BD2
:100020000F28F80B0E284A30F700F70B15280000B0
:100030000000800B0C28003405110130BF000720A0
:1000400005150130BF00072000348510051501306B
:10005000BF000720383086001C20013086001C209D
:10006000033086001C200F3086001C208A110829CE
:10007000851005150130BF000720013086001C20C7
:100080000F3086001C208A11092933088400430898
:100090008000840A8001B30A00340408C2003C0EC8
:1000A000F038BE00BE07E23EBF00323EC1003C0851
:1000B0000F39BF07BF07C107E93EC000C007C0072F
:1000C0003B0E0F39C007C107C00DC10DC109C10DDD
:1000D0003B080F39C107BE0D0730BD000A30C1070C
:1000E000C003031C6F28C007BF03031C7328BF078E
:1000F000BE03031C7728BE07BD03031C7B283D30CD
:100100008400073042058407413004020319A42803
:100110000008F700031D9228421AA228C219942849
:10012000203095280830C2003030F707BC010408A1
:10013000BB007708BD007708C30045203B0884005A
:100140003D08F700840A84280008F7003030F707DC
:100150007708C30045208A111229BC013B083C07DF
:10016000840080080319C4283B083C078400000869
:10017000BD003D08BE0085143E0886001C200130ED
:10018000BF000720BC0AAE288A11152984011F3040
:10019000830583161F08C0399F009B010730831217
:1001A0009F00B301F830831685008601083098005F
:1001B0009F019F1783129F151F169F121F139F13D6
:1001C0001F14B501B4011F1500301F190130013C87
:1001D0000319E428003083161E078312B4001E089A
:1001E000B5000318B50A83161E088312860008306E
:1001F000BB00FA30BF000720BB0BF9281E088600A1
:100200000830BB00FA30BF000720BB0B02292528AD
:1002100038283630B300103084003508BC0034086C
:10022000BB004D283630BB00AD280830BB00FA308B
:0C023000BF000720BB0B1729E328630068
:040000008A01032846
:00000001FF
